:1000000012C0189518951895189518951895189563
:100010001895189518951895189518951895189578
:100020001895189518958FED8DBFC0ECE0EC4E2E0D
:10003000DD275D2EEEE7F0E0A0E6B0E088278D93A7
:100040003197E9F784B7082E877F84BF8FE181BDA0
:1000500087E081BDE0D166248FEF81BB80E082BB69
:100060008CE021D2BF98ACE69C9197FF04C0B79971
:100070000EC09F779C93B79B0AC089E19F939927F5
:10008000A8D29F91B79B03C090689C9382D1A9D1BD
:10009000E8E4F7E09ED1E2E0F0E0B4D180E08093C4
:1000A0006A00A2E6BAD280E08093660080E0809386
:1000B0006B0097D1E8E5F7E08CD164D2A0E60C9311
:1000C00000916000003109F401C005D084E690E0A1
:1000D00080D2F3CFC5CF8FEF87BB939A84E690E0B1
:1000E00078D2939882E390E074D2EEE5F2E0A0E655
:1000F0008C919927A1E68CD200916A00013009F019
:1001000001C037C000916A00023009F001C05BC035
:10011000009161000B3009F017C034D2A0E60C93B7
:1001200000916000083009F001C0F7CF8FEF87BB66
:1001300058D1E6E6F7E04DD1AAE68C918F5F8C931B
:1001400080E0809366000895009161000C3009F012
:100150000FC0EAE0F0E0A4E194E0EFD2A2E60D9156
:100160001D912D913C9164D209F001C0D7C07DC092
:100170003DC0009161000C3009F024C08FEF87BBB7
:10018000EAE0F0E0A4E194E0D8D2A2E60D911D915E
:100190002D913C914DD209F401C067C0A2E63DD239
:1001A00080E08093660080E080936B00AAE68C91EB
:1001B0008F5F8C9316D188EC90E00BD2E6E7F7E0E6
:1001C00008D1089513C0009161000C3009F00EC0F1
:1001D0008FEF87BBEAE0F0E0A2E694E07BE79CD2F9
:1001E00000D1E6E8F7E0F5D088D058CFA6E68C91AC
:1001F0008F5F8C930091660044E0040FABE60C9394
:100200008FEBABE61C91FCD0E6E9F7E0E2D0009181
:100210006600083010F009F001C001C026C0A2E657
:100220000D911D912D913C914AE050E060E070E00D
:100230005AD1A2E60D931D932D933D93A2E60D9105
:100240001D912D913C91A1E64C915527662777276A
:10025000EAD1A2E60D931D932D933D9308950C09C9
:1002600006030A0805020B070401939ABAD0E8E9CD
:10027000F7E0AFD0E3E0F0E0C5D09398A9E68C9129
:100280008F5F8C9300916900033009F035C08CE3D7
:10029000809367004091670001E0041710F009F0B7
:1002A00027C08FEB13E0ACD0E6EAF7E092D08FEBFB
:1002B00019E0A6D0009167000A3008F003C0EEEA0A
:1002C000F7E087D0A8EAB0E0E7E6F0E0D3D179D054
:1002D0008FEB1BE095D0E0EBF7E07BD0E1E0F0E0C6
:1002E00091D08091670081508093670008F0D2CF51
:1002F00080E08093690001D0D1CE84E690E069D19E
:10030000939A88EC90E065D1939888EC90E061D165
:10031000939A88EC90E05DD19398089580E0809363
:100320006900E9E0F0E0A7E605D2009167000D3C26
:1003300008F00CC056D0E6EBF7E04BD050D0E8EC1C
:10034000F7E047D085B7816285BF889580916700C7
:10035000815080936700E9E0F0E0A7E67BE7D9D120
:1003600084E190E036D13DD0E6E8F7E032D0C5DF59
:1003700036D0EAEDF7E02DD08CE291E02AD1949AC4
:10038000E2E0F0E03FD094982CD0E1E0F0E03AD009
:1003900085CE27D0B79901C013C0EAE0F0E002EDA6
:1003A00014E020E030E0A0E1BB2794E07BE7B4D18B
:1003B000A4DF17D0E8EEF7E00CD0E3E0F0E022D0C5
:1003C0000895A8EAB0E08D91882311F066D0FBCFA4
:1003D00008950ED1802D11F060D0FBCF089580ECF0
:1003E00062C081E060D014D080E85DC08FE721302A
:1003F00039F08FEB223021F08FE8233009F08FECB9
:10040000810F51C088EE93E0E4D03197D9F7089579
:1004100083E09927DEC08AEF90E0DBD0BB9ABA9ADE
:10042000B99AB89A8E9A8D9A959885E090E0D1D035
:100430009698C398C298C19AC09A969AEF93FF93E0
:10044000E5E1F0E096D0FF91EF919698BFD0969AB3
:10045000EF93FF93E5E1F0E08CD0FF91EF91969858
:10046000B5D0969AEF93FF93E5E1F0E082D0FF914B
:10047000EF919698ABD0C098969AEF93FF93E5E1F1
:10048000F0E077D0FF91EF919698A0D088E20BD062
:100490008EE009D086E007D00895959A829505D020
:1004A00004D094D008959598F9CF859510F4C09A0A
:1004B00001C0C098859510F4C19A01C0C198859576
:1004C00010F4C29A01C0C298859510F4C39A01C075
:1004D000C398969AEF93FF93E5E1F0E04AD0FF913D
:1004E000EF919698089522D006D000FC01D008958F
:1004F00028D030D00895842F952FA62FB72F4427CA
:10050000552766277727F1E2889409C020F4480F21
:10051000591F6A1F7B1F76956795579547953795A5
:10052000279517950795FA9589F708950024E8947B
:1005300077FF02C006D0689400F809D010F80124B3
:10054000089512D04F5F5F4F6F4F7F4F0895E8942B
:1005500037FF089500951095209530950F5F1F4F38
:100560002F4F3F4F68940895409550956095709532
:1005700008953197F1F70895689462F80895E89422
:1005800062F8089500E18FEF88BB8FE087BB80EFB2
:1005900088BB88E28A95F1F7B49B00E0B59B04E044
:1005A000B69B08E0B79B0CE080EF87BB8FE088BB71
:1005B00088E28A95F1F78827B09B80E0B19B81E0C3
:1005C000B29B82E0B39B83E0080F089581E090E046
:1005D00000C0EF93FF93EE27E82BE92B31F0EAEF11
:1005E000F0E03197F1F70197D1F7FF91EF9108957E
:1005F000C89531960020089591E005C092E003C0AF
:1006000094E001C098E0F4DF0D929A95E1F7089527
:10061000E80FF91FF1CF82E001C084E099279D9394
:100620008A95E9F70895040F151F261F371F0895AF
:1006300004171507260737070895000F111F221FFB
:10064000331F089500951095209530950F5F1F4F2B
:100650002F4F3F4F0895019110810EC001911191CC
:10066000219130810BC00191108117FF05C03FEF30
:100670002FEF04C0008111272227332737FF03C043
:10068000E1DF8DE28D93CF93DF93CF92DF92EF92F4
:10069000AA24BB24CC24DD24EE2440E2CAE0DD27DA
:1006A00055E093E38881890F87FD9F7083FD907FDC
:1006B000891B89935A95A9F7C0DFAA1CBB1CCC1CC7
:1006C000DD1CEE1C4A9551F7E894EFE0FF2782917C
:1006D0000ED0EB30E0F71EF068948A2D0CD08827FE
:1006E0008D93EF90DF90CF90DF91CF910895982F69
:1006F000829501D0892F8F70805D26F0803309F4B8
:10070000089568948D930895E199FECFEEBB3196DC
:10071000089591E001C092E07B3751F47FB7F894DF
:10072000F3DF8D918DBBE29AE19A9A95C9F77FBF6D
:100730007727089591E001C092E0E6DFE09A8DB35B
:100740008D939A95D1F708955757572E4156522EAB
:10075000344D472E434F4D00202020456E74657266
:1007600020636F64650020456E746572206F6C6451
:1007700020636F64650020456E746572206E657736
:1007800020636F64650020436F6465206163636567
:100790007074656400002A00202020436F64652087
:1007A00077726F6E6700576169743A2000003000FD
:1007B000207365630000212044454D4F204558506B
:1007C000495245442021000047534D3A2B333836D7
:1007D0003430383332313739000020202020556E34
:1007E0006C6F636B65640000436F64652069732000
:0607F00031323334000039
:00000001FF
